:0200000480007A
:100000006F008004732F2034930F80006308FF0378
:10001000930F90006304FF03930FB0006300FF038E
:10002000130F000063040F0067000F00732F2034CC
:1000300063540F006F00400093E19153171F0000BD
:1000400023223FFC6FF09FFF732540F163100500F2
:10005000970200009382020173905230735000188F
:10006000970200009382020273905230B702008020
:100070009382F2FF7390023B9302F0017390023A75
:1000800097020000938282017390523073502030A7
:1000900073503030735040309301000097020000DD
:1000A000938282F673905230130510001315F501F8
:1000B000634C05000F00F00F930110009308D0056A
:1000C000130500007300000093020000638E02001D
:1000D00073905210B7B20000938292107390223046
:1000E00073232030E39A62F47350003097020000CB
:1000F0009382420173901234732540F173002030D3
:10010000930000001301000033972002930E0000BB
:1001100093012000631AD74B9300100013011000C5
:1001200033972002930E000093013000631ED749DD
:10013000930030001301700033972002930E0000EB
:10014000930140006312D749930000003781FFFFFD
:1001500033972002930E0000930150006316D74797
:10016000B70000801301000033972002930E0000B7
:1001700093016000631AD745B700008013010000A7
:1001800033972002930E000093017000631ED74343
:10019000B7B0AAAA9380B0AA370103001301D1E730
:1001A00033972002B70EFFFF938E1E089301E001E4
:1001B000631CD741B70003009380D0E737B1AAAAE8
:1001C0001301B1AA33972002B70EFFFF938E1E08CA
:1001D0009301F001631AD73FB70000FF370100FF1A
:1001E00033972002B70E010093010002631ED73D32
:1001F0009300F0FF1301F0FF33972002930E0000ED
:10020000930110026312D73D9300F0FF1301100019
:1002100033972002930EF0FF930120026316D73B21
:10022000930010001301F0FF33972002930EF0FFAC
:1002300093013002631AD739B700D0003701B000FC
:10024000B3902002B79E0000938E0EF093018000C1
:10025000639CD037B700E0003701B0003391200233
:10026000B7AE0000938E0EA093019000631ED135AF
:10027000B700D000B3901002B7BE0000938E0E906E
:100280009301A0006392D03513020000B700D000A4
:100290003701B00033972002130307001302120046
:1002A00093022000E31452FEB79E0000938E0EF0DE
:1002B0009301B000631AD33113020000B700E000CD
:1002C0003701B0003397200213000000130307002A
:1002D0001302120093022000E31252FEB7AE000098
:1002E000938E0EA09301C0006310D32F1302000061
:1002F000B700F0003701B000339720021300000070
:1003000013000000130307001302120093022000E1
:10031000E31052FEB7AE0000938E0E509301D00052
:100320006314D32B13020000B700D0003701B000D4
:10033000339720021302120093022000E31652FEAC
:10034000B79E0000938E0EF09301E000631ED72746
:1003500013020000B700E0003701B00013000000F6
:10036000339720021302120093022000E31452FE7E
:10037000B7AE0000938E0EA09301F0006316D72550
:1003800013020000B700F0003701B00013000000B6
:100390001300000033972002130212009302200082
:1003A000E31252FEB7AE0000938E0E50930100018F
:1003B000631CD72113020000B700D0001300000017
:1003C0003701B0003397200213021200930220007D
:1003D000E31452FEB79E0000938E0EF093011001BD
:1003E0006314D71F13020000B700E00013000000E1
:1003F0003701B000130000003397200213021200EF
:1004000093022000E31252FEB7AE0000938E0EA0BE
:1004100093012001631AD71B13020000B700F000FC
:1004200013000000130000003701B00033972002D2
:100430001302120093022000E31252FEB7AE000036
:10044000938E0E50930130016310D71913020000F0
:100450003701B000B700D00033972002130212001A
:1004600093022000E31652FEB79E0000938E0EF01A
:1004700093014001631AD715130200003701B00041
:10048000B700E000130000003397200213021200AF
:1004900093022000E31452FEB7AE0000938E0EA02C
:1004A000930150016312D713130200003701B0000B
:1004B000B700F00013000000130000003397200283
:1004C0001302120093022000E31252FEB7AE0000A6
:1004D000938E0E50930160016318D70F1302000032
:1004E0003701B00013000000B700D000339720029E
:1004F0001302120093022000E31452FEB79E000084
:10050000938E0EF0930170016310D70D130200005B
:100510003701B00013000000B700E0001300000036
:10052000339720021302120093022000E31252FEBE
:10053000B7AE0000938E0EA0930180016316D70919
:10054000130200003701B000130000001300000088
:10055000B700F0003397200213021200930220002C
:10056000E31252FEB7AE0000938E0E50930190013D
:10057000631CD705B700007C33111002930E0000F6
:100580009301A0016312D105B700008033910002EE
:10059000930E00009301B0016318D103B310000261
:1005A000930E00009301C0016390D003B7001002C6
:1005B0003701200233902002930E00009301D001F6
:1005C0006314D001631030020F00F00F638001004C
:1005D0009391110093E111009308D0051385010058
:1005E000730000000F00F00F930110009308D00576
:0C05F0001305000073000000731000C031
:1010000000000000000000000000000000000000E0
:1010100000000000000000000000000000000000D0
:1010200000000000000000000000000000000000C0
:1010300000000000000000000000000000000000B0
:081040000000000000000000A8
:040000058000000077
:00000001FF
